S01700006F70656E626C745F786D63343730302E73726563A7
S31508000000C899FE1F79500008C9500008CD5000084D
S31508000010D1500008D5500008D9500008000000004B
S31508000020000000000000000000000000DD5000088D
S31508000030E150000800000000E5500008E9500008FB
S31508000040ED500008F1500008F5500008F950000876
S31508000050FD50000801510008055100080951000823
S315080000600D5100080000000000000000000000001C
S315080000701151000800000000155100081951000828
S315080000801D51000821510008255100082951000872
S315080000902D51000831510008355100083951000822
S315080000A03D510008415100084551000849510008D2
S315080000B04D51000851510008555100085951000882
S315080000C05D51000861510008655100086951000832
S315080000D06D510008715100087551000879510008E2
S315080000E07D51000881510008855100088951000892
S315080000F08D51000891510008955100089951000842
S315080001009D510008A1510008A5510008A9510008F1
S31508000110AD510008B1510008B5510008B9510008A1
S31508000120BD510008C1510008C5510008C951000851
S31508000130CD510008D1510008D5510008D951000801
S31508000140DD510008E1510008E5510008E9510008B1
S31508000150ED510008F1510008F5510008F951000861
S315080001600000000000000000000000000000000081
S31508000170FD510008015200080552000809520008FE
S315080001800D520008115200081552000819520008AD
S315080001901D5200082152000825520008295200085D
S315080001A02D5200083152000835520008395200080D
S315080001B03D520008415200084552000849520008BD
S315080001C04D5200085152000855520008595200086D
S315080001D05D520008615200086552000800000000E0
S315080001E0695200086D5200087152000875520008DD
S315080001F079520008000000007D5200080000000047
S31508000200C2788A18DFF83833DA7083780A0092B22F
S31508000210120AD218DFF828339A704278DFF82033AA
S315080002205A700078DFF818231070DFF81403827804
S31508000230080080B2000A80B2824212DADFF80003B0
S315080002404078401CDFF8F8225070DFF8F402407856
S31508000250002806D1DFF8E8020078401CDFF8E02223
S315080002601070DFF8DC02C07889B201F0FF0188421D
S315080002701EDADFF8CC028078401CDFF8C4128870DA
S31508000280DFF8BC028078002812D1DFF8B402407883
S31508000290401CDFF8AC124870DFF8A402407800284A
S315080002A006D1DFF89C020078401CDFF8941208702B
S315080002B0704710B492B20A44531E0BE00A78120231
S315080002C04C78121910180400A4B292B2944200D2C3
S315080002D0401C891C9942F1D3994208D109780A022F
S315080002E01018010089B292B2914200D2401C80B225
S315080002F010BC704780B51422DFF848120020FFF7BB
S31508000300D8FF80B2002802D14FF6FF7002E080B213
S3150800031001F036FA80B202BD10B5DFF82C12097C5E
S315080003200902DFF82422527C8918B1F1140454FA20
S3150800033080F00822DFF8141280B2FFF7BAFF220015
S3150800034092B2DFF80C1280B2FFF7B3FF80B2002832
S3150800035002D14FF6FF7002E080B201F011FA80B2C6
S3150800036010BD80B50620FFF7D7FF02BD0020DFF8D5
S31508000370E41108700EE00020DFF8DC11DFF8D42164
S31508000380127821F81200DFF8CC010078401CDFF85B
S31508000390C4110870DFF8BC0100780028EBD00020F3
S315080003A06C4908700CE000206C496A4A1278682388
S315080003B05A431144487667480078401C65490870D6
S315080003C0644800780028EED04FF4806064490880BD
S315080003D00020604908700CE0002062495D4A1278E6
S315080003E040235A43114488805A480078401C59498A
S315080003F00870584800780028EED0704770B5040099
S315080004000D000CE0574853490978402251430844E7
S3150800041086885348008801F0B3F9864211D15048BE
S315080004200088401C4E4908804D480088B0F5FA4FB0
S3150800043003DB4FF480504A4908800020454908707C
S3150800044004E044480078401C424908704148007856
S315080004500028D7D0002600203E49087004E03D4811
S315080004600078401C3B4908703A48007800280FD1AC
S315080004703C48384909784022514308448088002876
S31508000480EDD13848334909784022514300EB01063B
S31508000490002E01D1002018E031480088304909882B
S315080004A089B2090A51EA0020B080F580002C05D1EE
S315080004B004210022300001F097F903E020883080FB
S315080004C06088708040203072300070BD0021214A5B
S315080004D0117004E01F490978491C1E4A11701D490C
S315080004E0097800290CD11C491A4A127831F81210D9
S315080004F00029EFD11849174A127821F81200FFE7A8
S31508000500704780B5010089B2174800680830FFF7C0
S3150800051077FE0B480078144909680872084840783D
S31508000520114909684872064880780F49096888722F
S315080005300348C0780C490968C87201BD000000006C
S315080005408C91FE1FB280FE1FA480FE1FBE80FE1F78
S31508000550C680FE1FA891FE1F9A91FE1FF08EFE1FF1
S315080005609E91FE1F8890FE1F8091FE1F10B5DFF832
S31508000570141E0C68C0B2042806D1DFF83C0E0088A9
S31508000580002840F061821DE0DFF8301EDFF8302ECB
S315080005901160DFF82C1E0968DFF8282E1160C0B23A
S315080005A0032818D1607E10F00F0003280AD1208A8C
S315080005B0002807D10820DFF8281E087001F0E1F9A5
S315080005C000F0A9BF0020DFF81C1E08800020DFF815
S315080005D0101E087010BDC0B2022840F0D180DFF8A6
S315080005E0080EC078401CDFF8001EC870DFF8F80D4A
S315080005F0C07800281ED1DFF8F00D8078401CDFF89F
S31508000600E81D8870DFF8E00D8078002812D1DFF841
S31508000610D80D4078401CDFF8D01D4870DFF8C80DAB
S315080006204078002806D1DFF8C00D0078401CDFF8B6
S31508000630B81D08700020DFF8AC1D08800020DFF820
S31508000640781D0880607E072802D0607E052808D1BC
S31508000650A07E401CA076A07E782801D10020607676
S31508000660B0E7607E0028FBD0208A00287AD0A07EDA
S31508000670411EA176C0B20028F2D1E07E082808D033
S31508000680607E022802D0607E012810D1E07E05280F
S315080006900DD1002060768020DFF8441D087001F037
S315080006A070F91420DFF8B01D81F82F00B0E2E07E63
S315080006B0052801DB042000E0E07E032111FA00F0A2
S315080006C0A076E07E401CE076607E10F00F00C0B297
S315080006D001280AD0022835D0032839D004283FD06B
S315080006E006283DD008283BD0BAE71020DFF8681D59
S315080006F081F82F00DFF8600D90F82F0050F0020007
S31508000700DFF8541D81F82F000220DFF84C1D81F810
S3150800071036000420DFF8401D81F837000620DFF890
S31508000720381D81F838000A20DFF82C1D81F83900B9
S315080007302C20DFF8B01C08806020DFF81C1D81F82B
S315080007402E006EE20020DFF8101D81F82F00D1E799
S315080007500420DFF88C1C087001F013F900F01FBFA5
S3150800076000F074BE607E10F00F0003287FF478AFA7
S315080007700820DFF86C1C087001F003F900F0CBBE06
S31508000780C0B2052826D1DFF8040E00688088002844
S315080007901FD00020DFF8EC1B0860DFF8F40DDFF847
S315080007A0201C0860DFF8180C0068DFF8181C0860C1
S315080007B00020DFF8041C0880DFF8FC0B0088DFF84F
S315080007C0241C08800820DFF8181C087001F05DFC5E
S315080007D0D3E6F7E6DFF8800C807B45287FF4F2AE97
S315080007E0DFF8000C0088DFF8701C097C0902DFF8C6
S315080007F0682C527C8918884216DBDFF85C0C007C72
S315080008000002DFF8541C497C4018DFF8D81B088022
S31508000810DFF8440C007D3F21084204D1DFF8380C8C
S31508000820407D002801D0CDE6CCE6DFF8B80D00887B
S31508000830DFF8B41D0988884207D1DFF8A80D40887B
S31508000840DFF8A41D4988884210D0DFF80C0CC08B4D
S31508000850DFF8901D0988884207D1DFF8FC0B008C69
S31508000860DFF8801D4988884200D0ABE6FFF742FDD5
S315080008704FF6FF7188427FF4A5AEDFF8DC0BC07D2A
S31508000880062809D1FFF76DFD4FF6FF71884240F043
S315080008903D81DFF8584D3BE1DFF8BC0BC07D1128E0
S315080008A00CD1DFF8400B00881C38DFF8381B0880AD
S315080008B0DFF8080EDFF8D41C086048E0DFF8980B6C
S315080008C0C07D01287FF47EAEDFF88C0B90F82200FD
S315080008D008287FF477AE0020DFF87C1B81F8220019
S315080008E0DFF8740B808C4FF6F771884207DBDFF868
S315080008F0680B808C0930DFF8601B888406E0DFF817
S31508000900580B808C0830DFF8501B8884DFF8480BBA
S31508000910408BDFF8441BC883DFF83C0B808BDFF87D
S31508000920381B0884DFF8BC0C0088DFF82C1B4883CA
S31508000930DFF8B00C4088DFF8201B888300F019BF69
S31508000940DFF8480C00684030DFF8401C0860DFF824
S315080009503C0C0068DFF8681D884274D2DFF82C0C5E
S31508000960006880880028EBD0DFF8EC0A808CDFF876
S315080009701C1C096889888842E2D1DFF8100C0068D7
S31508000980C08800280FD0DFF8D00A408CDFF8FC1B9F
S315080009900968C988884206D0DFF8F00B0068C08865
S315080009A0B0F58A4FCCD1DFF8E40B00680088DFF891
S315080009B0381C0988884208D1DFF8D00B00684088BF
S315080009C0DFF8241C4988884223D0DFF8C00B00686A
S315080009D00088DFF8A81D0988884208D1DFF8AC0B23
S315080009E000684088DFF8941D4988884211D0DFF8EE
S315080009F0680A408BDFF8941B0968098888429FD1EA
S31508000A00DFF8540A808BDFF8841B09684988884216
S31508000A1096D10020DFF86C1908600220DFF8C019AB
S31508000A200870DFF86C0BDFF898190860DFF8900992
S31508000A300068DFF8901908600020DFF87C19088044
S31508000A4001F023FB99E5BDE5DFF86C0900881C3049
S31508000A50DFF890190880DFF88C09008880B2000A50
S31508000A60DFF8F4190874DFF87C090088DFF8E8195C
S31508000A704874DFF8180B0068007ADFF8DC19887507
S31508000A801120DFF8D419C875DFF82C09008808305A
S31508000A90DFF824190988083189B2090A51EA0020C1
S31508000AA0DFF8B419C8840020DFF8AC190885DFF828
S31508000AB0DC0A00688088DFF8A0194884DFF8CC0AC9
S31508000AC00068C088DFF890198884DFF8180B00885A
S31508000AD0DFF884194883DFF80C0B4088DFF87819AB
S31508000AE08883DFF8A80A00680088DFF86C19C883CD
S31508000AF0DFF8980A00684088DFF85C190884DFF890
S31508000B00BC08DFF8BC18086000F00FBE5AE5683468
S31508000B10DFF8D80AA042C0F0DF80607E0028F6D051
S31508000B20DFF83409808CA1888842F0D1DFF82809DB
S31508000B30408CE1888842EAD1DFF81C09408B21887D
S31508000B408842E4D1DFF81009808B61888842DED1BB
S31508000B50DFF8300804600020DFF884180870DFF832
S31508000B60F80890F82F00400700F1CD82DFF8E80872
S31508000B7090F82E00C0B200098000DFF8381C087013
S31508000B80DFF860080088DFF82C1C0978401A14384A
S31508000B90DFF850180880607E10F00F00022808D190
S31508000BA0DFF8B40890F82F0010F03F00122800F084
S31508000BB0B382DFF830080088002807D1DFF89808E4
S31508000BC090F82F000321084200F0A682DFF8880873
S31508000BD090F82600217A884215D1DFF87C0890F82B
S31508000BE02700617A88420ED1DFF86C0890F8280051
S31508000BF0A17A884207D1DFF8600890F82900E17ADF
S31508000C00884200F089821020DFF84C1881F82F00FE
S31508000C102820DFF8D01708805020DFF83C1881F824
S31508000C202E00207ADFF8301881F82A00607ADFF87B
S31508000C30281881F82B00A07ADFF81C1881F82C00F8
S31508000C40E07ADFF8141881F82D00207BDFF8081801
S31508000C5081F82600607BDFF8001881F82700A07B62
S31508000C60DFF8F41781F82800E07BDFF8EC1781F845
S31508000C7029000620DFF8E017C875A088DFF8D8171E
S31508000C804884E088DFF8D0178884DFF85809008898
S31508000C90DFF8C4174883DFF84C094088DFF8B8172F
S31508000CA088832088DFF8B017C8836088DFF8A8171C
S31508000CB00884607EC00640F111850020DFF8981789
S31508000CC081F83100DFF8900790F83100DFF88817CF
S31508000CD081F8300000F00ABDDFF87C0790F82F0095
S31508000CE010F03F00022806D0DFF86C0790F82F00B6
S31508000CF0400729D566E4DFF86007808CDFF8B81A64
S31508000D0008800020DFF8AC1A087006E0DFF8A40AAD
S31508000D100078401CDFF89C1A0870DFF8980A0078FB
S31508000D200028E1D1DFF8900A0088DFF8901ADFF88A
S31508000D30842A127831F812108842E7D1002400205C
S31508000D40DFF8701A0870F0E01420DFF80C1781F845
S31508000D502F002820DFF88C1608805020DFF8F816B8
S31508000D6081F82E00DFF8F00690F82900DFF8441A1B
S31508000D700870DFF8E40690F82D00DFF8DC1681F835
S31508000D802900DFF8300A0078DFF8CC1681F82D0044
S31508000D90DFF8C40690F82800DFF8181A0870DFF89C
S31508000DA0B80690F82C00DFF8B01681F82800DFF8AE
S31508000DB0040A0078DFF8A01681F82C00DFF89806F8
S31508000DC090F82700DFF8EC190870DFF88C0690F821
S31508000DD02B00DFF8841681F82700DFF8D809007899
S31508000DE0DFF8741681F82B00DFF86C0690F82600F9
S31508000DF0DFF8C0190870DFF8600690F82A00DFF8F7
S31508000E00581681F82600DFF8AC090078DFF848168E
S31508000E1081F82A00DFF8400690F82D00401CDFF81C
S31508000E20381681F82D00DFF8300690F82D000028D6
S31508000E3026D1DFF8240690F82C00401CDFF8181697
S31508000E4081F82C00DFF8100690F82C00002817D13E
S31508000E50DFF8040690F82B00401CDFF8FC1581F833
S31508000E602B00DFF8F40590F82B00002808D1DFF8EE
S31508000E70E80590F82A00401CDFF8DC1581F82A00FE
S31508000E80DFF8D405408CDFF830190880DFF8C8058C
S31508000E90808CDFF8C4154884DFF81C090088DFF861
S31508000EA0B8158884DFF8B005408BDFF8AC15C88321
S31508000EB0DFF8A405808BDFF8A0150884DFF824077F
S31508000EC00088DFF894154883DFF818074088DFF8AC
S31508000ED08815888300F00ABCDFF81007DFF8D418F5
S31508000EE00978682251430844407E072816D1002C09
S31508000EF00BD0A07EDFF8F416DFF8B828127868233E
S31508000F005A431144897E884208D2DFF8E006DFF8A2
S31508000F10A41809786822514300EB0104DFF8940805
S31508000F200078401CDFF88C180870DFF8880800780D
S31508000F30002813D1DFF8B406DFF878180978682294
S31508000F4051430844407E0028C6D1DFF8A006DFF8E2
S31508000F50641809786822514300EB0104002C3FF419
S31508000F6031ABDFF8200404600320A076A07E20764B
S31508000F700020A0750420E0750020E076DFF8D8048C
S31508000F80808CA080DFF8D004408CE080DFF8C804AD
S31508000F90408B2080DFF8C004808B6080012060765B
S31508000FA0DFF8440400782073DFF83C044078607367
S31508000FB0DFF834048078A073DFF82C04C078E07377
S31508000FC001202082DFF8900490F82900E072DFF80B
S31508000FD0880490F82800A072DFF87C0490F82700AF
S31508000FE06072DFF8740490F8260020720120FFF77B
S31508000FF088FADFF8640490F82E0010F0F000512803
S31508001000FFF673AB0020DFF8AC17087006E0DFF8D0
S31508001010A4070078401CDFF89C170870DFF89407CF
S315080010200078DFF8341491F82E10C9B20909C9B24C
S31508001030491FB0EB810FBFF658ABDFF81C04DFF889
S3150800104074170978084490F83600DFF874170870A2
S31508001050DFF86C07007800283FF447ABDFF8600735
S3150800106000780128D3D0DFF85807007802282FD156
S31508001070DFF8E403DFF83C170978084490F83700EE
S31508001080042825D1DFF8D003DFF8281709780844A3
S3150800109090F83800DFF8C013DFF8182712781144E3
S315080010A091F8391051EA0020DFF80C170880DFF8AC
S315080010B00807008840F20B61884202DB40F20A60AA
S315080010C002E0DFF8F40600886082A082FFF70DBB15
S315080010D0DFF88403DFF8DC160978084490F837004F
S315080010E000283FF402ABDFF8CC060078DFF8681377
S315080010F0DFF8C0261278114491F837100818DFF87F
S31508001100B41608708AE7002060762020B449087073
S3150800111000F037FCFFF756BACF4890F82F00C00604
S315080011205FD5208A00285CD0218A14F10C00FFF7CD
S3150800113067F8C94890F82A00DFF8881609788842BF
S315080011404FD1C54890F82B00DFF8781649788842C1
S3150800115047D1C14890F82C00DFF86816897888428C
S315080011603FD1BD4890F82D00DFF85816C978884257
S3150800117037D1DFF8500600782073DFF84806407844
S315080011806073DFF840068078A073DFF83806C07809
S31508001190E073E07E00281DD194F9180094F91A101E
S315080011A0401AA17DC9B2B0EBD100A17D4118A17545
S315080011B040B2002801D540B24042E17DC9B2B0EB49
S315080011C09100E17D4018E075A07DC0B2E17D11EB8C
S315080011D0D0002076012082490870207EA076002063
S315080011E02082607E10F00F00C0B2012813D0C0F034
S315080011F07382032800F0FA802ED3052800F03B827C
S31508001200C0F00482072800F05D82C0F05D820828DD
S3150800121000F0F08160E272480078C0071AD5032012
S31508001220607640206E490870002020826D4800884C
S31508001230002809D06A48007850F00200684908700A
S3150800124068480088FFF75DF900205B49088000F0D0
S3150800125098FB60E1FFF7B6B961480078C00740F12E
S31508001260B3807D4890F82F0010F03F00122840F018
S31508001270AB80794890F82E0010F0F000512827DB53
S315080012800020DFF83015087006E0DFF8280500783A
S31508001290401CDFF820150870DFF8180500786E493D
S315080012A091F82E10C9B20909C9B2491FB0EB810FCE
S315080012B00EDA6948DFF8FC140978084490F8360015
S315080012C0DFF8FC140870DFF8F8040078002822D14B
S315080012D003206076604890F8260020725E4890F8F1
S315080012E0270060725C4890F82800A0725A4890F867
S315080012F02900E0720120FFF704F9422038490870F6
S315080013000020208200203749088000202A490880CA
S3150800131000F037FBFFE0DFF8A80400780128B4D016
S31508001320DFF89C04007802282ED14B48DFF8841495
S315080013300978084490F83700042825D14648DFF88C
S3150800134074140978084490F838004349DFF864248F
S315080013501278114491F8391051EA0020DFF8581430
S315080013600880DFF85404008840F20B61884202DBEB
S3150800137040F20A6002E0DFF8400400886082A0823A
S31508001380A6E700BF8091FE1F3348DFF828140978C6
S31508001390084490F8370000289AD0DFF81804007837
S315080013A02D49DFF810241278114491F837100818DF
S315080013B0DFF8001408706FE79891FE1FDA80FE1FA9
S315080013C07891FE1F7C91FE1F20200549087000F0C9
S315080013D0D8FA0020DFF8F0130968487684E400BFDD
S315080013E0A791FE1F9691FE1F8891FE1F1A4890F836
S315080013F02F00C00732D5607EC0062FD4208A002869
S315080014007FF4E0A8DFF8C4030088401C80B2FFF729
S3150800141078F8DFF8BC03007850F01000DFF8B01356
S315080014200870DFF8A8030088002807D0DFF8A003B3
S31508001430007850F00200DFF89813087000F0A1FA5F
S3150800144001202082082060760020E07611200249DB
S3150800145081F82F00FFF7DCBBA480FE1FDFF87403BA
S3150800146090F82F00800621D5DFF86C030068DFF8B6
S31508001470641391F83410DFF85C2392F8352052EAA9
S3150800148001210844DFF850130860DFF8400300889C
S31508001490DFF8401391F83410DFF8382392F8352036
S315080014A052EA0121401ADFF824130880DFF81C03EA
S315080014B0008800280CD0607EC00609D4C44800788D
S315080014C050F00200C2490870C0480088FFF719F8B2
S315080014D0C04890F830000002BE4991F83110401813
S315080014E0B5490880A08AB4490988884203D3B24816
S315080014F00088002802D1A08AAF490880AE48008833
S315080015006082B34800780321084271D00020B349AD
S31508001510088000F036FAAE48007880060AD5002022
S31508001520AE490880002060761420AA4981F82F0069
S31508001530FFF76EBBA6480078C0060ED50020A7495F
S31508001540088001202082042060760020E0761120A1
S31508001550A04981F82F00FFF75BBBA0480088002848
S315080015601BD09B480078C00701D500202082208A1E
S3150800157000280FD1608A99490988884202D2608A70
S315080015809649088095480088208206E08491FE1FC7
S31508001590CE80FE1F208A914908800020E076904878
S315080015A000688D4908608D48008800280CD0208A7C
S315080015B0002809D0208A28308449088018208549BF
S315080015C081F82F00FFF728BB8148007880070FD5E0
S315080015D028207E49088010207E4981F82F00FFF7D1
S315080015E01BBB00BF6C91FE1FC0500008F08EFE1F8B
S315080015F0FEF7E8BF76480078C00706D50020607673
S3150800160010207349087000F0BCF965E06F4800883F
S31508001610002803D06D480088FEF773FF6D4890F8E0
S315080016202F00C00716D56A480078C00706D50720D8
S3150800163060760020A0760020208201E006206076F1
S315080016400120FEF75EFF10206149087000F099F945
S31508001650FFF7D9BA5E480078C00705D50520607639
S3150800166000202082FEF7AEBF5848008800287FF485
S31508001670CAAAFEF7A7BF55480088002803D05348D2
S315080016800088FEF73EFF534890F82F00C0070DD597
S31508001690072060760020A0760120FEF732FF102092
S315080016A04B49087000F06DF9FFF7ADBA4748008856
S315080016B000287FF4A8AAFEF785BF00BF8890FE1F02
S315080016C0C890FE1FFFF79FBA41480078C00703D5A8
S315080016D0072060760020A076FEF774BF06203D49F5
S315080016E081F830000A203B4981F831004020394909
S315080016F088753648008880B2000A36490874334827
S315080017000088344948740020324981F83500314848
S3150800171090F835002F4981F8340000202D49488675
S31508001720FEF71FFEC0432B49488645202949887382
S3150800173000202849C8730020264948752548407D59
S315080017402449087527480088401C264908802548EA
S31508001750008880B2000A1F498874224800881D49FB
S31508001760C87400201B490883FEF7C4FDC043194905
S315080017700883002016490870FEF72CBFBC500008E5
S31508001780010089B2090A51EA002080B2704710B5F3
S3150800179001290DDB114A118011490968884207D0D1
S315080017A00E490A880E490C680100200000F0B8FCB2
S315080017B010BD0000A891FE1FA091FE1F9A91FE1F62
S315080017C0A991FE1F8C91FE1F8091FE1F9691FE1F08
S315080017D0A791FE1FA480FE1F7891FE1F9891FE1FF9
S315080017E07C91FE1F9C91FE1F62F30F2262F31F423B
S315080017F0401810F0030308D0C91A1FD3DB0748BFE7
S3150800180000F8012D28BF20F8022D130030B4144625
S315080018101546103928BF20E93C00FAD8490728BFE1
S3150800182020E90C0048BF40F8042D890028BF20F89D
S31508001830022D48BF00F8012D30BC7047C91818BFE3
S3150800184000F8012DCB0728BF00F8012D70470000CE
S3150800185080B5AA480078002856D100F0F5FC00F0BB
S3150800186069FE10F5FA70A649086000F063FE00F5F7
S315080018701C501030A3490860FEF778FD0020ADF82B
S3150800188000000020ADF80200BDF800009E4908805F
S31508001890BDF802009C4948800020ADF800000020F1
S315080018A0ADF80200BDF8000098490880BDF80200AE
S315080018B0964948800020ADF800000020ADF80200E7
S315080018C0BDF8000092490880BDF80200904948809A
S315080018D04EF60300FEF7FAFD00F030FD8D4800F0E5
S315080018E083FD06218B4800F0ACFB00F0D2FB00F02C
S315080018F057FE42F21071884203D242F2107000F08D
S315080019004CFE01208449087001BD80B500207B4942
S31508001910087081480078002801D1FFF799FF01BDBA
S3150800192038B57D4A1278012A21D17C4A126812F10B
S315080019301C0422686260002206E092B2835C92B2BE
S3150800194004EB02052B72521C13000D00EDB29BB27C
S31508001950ADB2AB42F1D3C9B2081DA4F84800B4F839
S315080019604810201DFFF713FF2068401C206031BD7A
S3150800197080B569480078012801D100F03BF80020BD
S3150800198002BD10B56548006810F11C04644800786B
S31508001990400605D5012020600020A4F8480028E06C
S315080019A05F480078C00702D50020A4F848005C48C4
S315080019B00078400708D5B4F84800002804D0B4F8E1
S315080019C04810201DFFF7E3FE55480078800710D51C
S315080019D054480088001F41280BDA0020A4F8480064
S315080019E0514800684F490988091FC9B2001D00F00F
S315080019F015FE10BD10B500F004FD00282DD049498C
S31508001A0008804FF40060FFF7BBFE4849898980B219
S31508001A1081420ED10120FEF7A9FD42480088002820
S31508001A201BD001F059F900F000FD00203D4908805F
S31508001A3013E040F60600FFF7A3FE3C49898980B209
S31508001A4081420AD101F0DEF836480088002804D021
S31508001A5000F0EBFC00203349088000F06BFD2849B4
S31508001A600968884239D32648006810F5FA7024496F
S31508001A700860002415E02E48682101FB04F108449B
S31508001A80264908600220FEF771FD264800880028CE
S31508001A9006D001F021F900F0C8FC00202149088091
S31508001AA0641C002CE7D0002415E02248402101FBE5
S31508001AB004F10844204908600520FEF757FD194837
S31508001AC00088002806D001F007F900F0AEFC0020D7
S31508001AD014490880641C002CE7D000F02BFD094946
S31508001AE00968884208D30748006800F51C5010307A
S31508001AF00449086000F0AEFF10BD0000A180FE1F7B
S31508001B005C91FE1F6091FE1F6C91FE1F7491FE1F73
S31508001B107091FE1F4091FE1FA491FE1F8091FE1F2B
S31508001B20A791FE1F9691FE1F7891FE1FA480FE1FA7
S31508001B30F08EFE1F8890FE1F8491FE1F35220270CC
S31508001B40401C01220270401C0170401C704710B5F1
S31508001B50040036202070641C04202070641C0422B3
S31508001B60DFF87815200000F0DBFA201D10BD10B54F
S31508001B70040032202070641C04202070641C042297
S31508001B80DFF85C15200000F0CBFA201D10BD3721C8
S31508001B900170401C03210170401C01210170401C8A
S31508001BA003210170401C06210170401C7047FF216B
S31508001BB00170401C704738B50400012020700120D0
S31508001BC06070DFF820058069A0700020E0700422AC
S31508001BD0DFF81415251D280000F0A2FA0020208140
S31508001BE0802060810422DFF8041514F10C05280012
S31508001BF000F096FA0421002214F110052800FFF7D8
S31508001C00F3FD0421002214F114052800FFF7ECFD6A
S31508001C100421002214F118052800FFF7E5FDDFF876
S31508001C20C4048269DFF8BC04416914F11C05280064
S31508001C3000F076FADFF8AC048069D0F110010022D2
S31508001C40DFF8A0048069204410F11C052800FFF77E
S31508001C50CBFD4021002214F12C052800FFF7C4FD16
S31508001C608021002214F16C052800FFF7BDFD04222F
S31508001C70DFF87C14EC34200000F052FA31BD10B5C0
S31508001C80DFF8700404682000FFF795FF012114F1BE
S31508001C90F000FFF753FFFFF77AFFFFF788FFDFF83B
S31508001CA054140968411ADFF84C040068FFF76FFD01
S31508001CB010BD10B5DFF83C0404682000FFF77BFF71
S31508001CC0032114F1F000FFF739FFFFF740FFFFF794
S31508001CD04EFFFFF76CFFDFF81C140968411ADFF89E
S31508001CE014040068FFF753FD10BDF8B5060006EBAF
S31508001CF00104002509E00422B11CDFF8FC73380052
S31508001D0000F00EFA70783044861CA64234D2307839
S31508001D100128F0D003280AD0062810D0332820D06E
S31508001D20352814D0362814D0FF2822D0EAE7042212
S31508001D30B11CDFF8C873380000F0F2F9E2E70422B4
S31508001D40B11CDFF8BC73380000F0EAF9DAE7B578B9
S31508001D50D8E70422B11CDFF88473380000F0E0F9F4
S31508001D60D0E70422B11CDFF89C73380000F0D8F9DC
S31508001D70C8E72800C0B201E02800C0B2F2BD38B5F5
S31508001D80DFF8700304682078022823D10422DFF8DC
S31508001D905813201D01F082F800281BD1DFF84403F0
S31508001DA08269DFF84003416914F11C0001F076F8F6
S31508001DB000280FD1042214F11001DFF8245328005B
S31508001DC000F0AEF9DFF84003018814F1F000FFF7E0
S31508001DD08CFF00E0002032BD10B50120DFF80413A7
S31508001DE00988002916D040F20F12891A25D0491EF3
S31508001DF02CD0153960D0491E67D02F3900F0BB802A
S31508001E00491E00F0C180143900F0DC80491E00F03C
S31508001E10E28010E10120B34988704FF47A70B14925
S31508001E200861FFF72CFFAF480169B84801F067F869
S31508001E30002040F20F11AB4A1180C0B2002801D130
S31508001E400320FDE04FF48870A6490880B048007862
S31508001E50800706D4AD4801F059F8002801D10020C2
S31508001E60EEE0AB480078800707D5FFF788FF022821
S31508001E7003D102209B4988700EE09A4800694EF605
S31508001E806021884204DA974800694000954908614C
S31508001E90944880780228C4D14FF47A709149086131
S31508001EA0FFF707FF8F480169984801F028F80020D6
S31508001EB040F225118B4A1180C0B2002801D10320B7
S31508001EC0BEE04FF4937087490880914800788007F0
S31508001ED006D48E4801F01AF8002801D10020AFE098
S31508001EE08B480078800722D5FFF749FF05281ED1C1
S31508001EF003207C4988707B4800F0DCF87948008C20
S31508001F00FFF73EFC04047748408CFFF739FC04438E
S31508001F1064084FF47A7000FB04F0B0F1004F1CD24D
S31508001F204FF47A7000FB04F06E49086119E06D48B9
S31508001F30006942F2117188420ADA6A48006910F5A6
S31508001F407A7068490861674880780328A8D1D2E77B
S31508001F50002064490880002072E07FF00040614953
S31508001F60086160480169694800F0C9FF002040F22D
S31508001F7055115C4A1180C0B2002801D103205FE0E8
S31508001F804FF4AB7057490880604800F0BFFF00283F
S31508001F9001D1002054E00220524988704FF47A702B
S31508001FA05049086100F075F800F0B8F8FFF781FEAF
S31508001FB04C480169554800F0A2FF00204FF4B5715E
S31508001FC0484A1180C0B2002801D1032038E040F207
S31508001FD06B10444908804E480078800706D44B4861
S31508001FE000F094FF002801D1002029E04848007835
S31508001FF080070AD5FFF7C3FE052806D1032039490D
S315080020008870384800F056F878E73648006942F292
S31508002010117188420ADA3348006910F57A70314935
S315080020200861304880780328C0D1EAE700202D49A6
S315080020300880002004E0002000202A4908800220A9
S3150800204010BD80B5274A5061264881610020254980
S3150800205088704FF6FF70ADF800004FF6FF70ADF8C8
S3150800206002004FF486416846FEF7C8F91D494860E4
S315080020701C484068002804D04FF48840194949682C
S31508002080888000201749088001BD80B5FFF7A4FEA7
S3150800209001BD81B00020ADF800000020ADF80200B7
S315080020A0BDF8000011490880BDF802000F494880B4
S315080020B001B07047818C0D4A1180C18C0B4A518042
S315080020C0018D144A1180418D124A5180018E124A9F
S315080020D01180408E1049488070470000E490FE1F2A
S315080020E0EC90FE1FC890FE1FB45000086C91FE1FAE
S315080020F0B85000087891FE1FF090FE1FF890FE1F5A
S31508002100F490FE1FE890FE1F9691FE1FD090FE1FCA
S31508002110A791FE1F7491FE1F7091FE1F7047000065
S3150800212062B38B0708D0521E11F8013B00F8013B39
S3150800213000F024808B07F6D1830740F0208000BF8B
S31508002140103A07D330B4B1E83810103AA0E838107E
S31508002150F9D230BC530724BFB1E80810A0E808102C
S3150800216044BF51F8043B40F8043BD20724BF31F87A
S31508002170022B20F8022B44BF0B7803707047083AED
S3150800218007D3B1E80810083A40F8043B40F804CBF6
S31508002190F7D25307E4E70000CF48016070470168AB
S315080021A0096831F4801100680160704703681B688C
S315080021B033F4904309B2194312B21143006801601F
S315080021C07047416990F8260040010858C00FC0B210
S315080021D07047016841F21802895851F002010268F5
S315080021E041F21803D1500168096851F004010068EA
S315080021F001607047016841F21802895851F400518C
S31508002200026841F21803D1500168096851F00801C3
S315080022100068016070470221026841F21403D15038
S315080022200021006841F2040281507047416990F824
S3150800223026004001084480687047426990F82600E5
S315080022404001104441607047E0B55FF4803001906A
S3150800225000208DF800006A460921A04800F064FEB7
S3150800226000208DF800006A4604219D4800F05CFEB7
S3150800227000208DF800006A460221994800F054FEB5
S3150800228000208DF800006A460321954800F04CFEB0
S3150800229000208DF8080088208DF800006A46052180
S315080022A08F4800F041FE00208DF8080088208DF840
S315080022B000006A4608218A4800F036FE00208DF89C
S315080022C0080088208DF800006A460921844800F035
S315080022D02BFE00208DF800006A4608217F4800F092
S315080022E023FE00208DF8080088208DF800006A4635
S315080022F007217B4800F018FE00208DF800006A468A
S315080023000021774800F010FE01220021744800F0F1
S3150800231093FE5FF080618908890031F00C01022084
S3150800232060F30921022060F38B2131F4404101203A
S3150800233060F397516B48FFF72FFF07BD1CB5694837
S3150800234000F0AFFE6748FFF72AFF00F0F3F800F544
S315080023509854883401E001F03BF80021614801F007
S31508002360B0F8002803D100F0E5F8A042F3D35E4A9E
S3150800237000215C4801F059F84FF400624FF480419F
S315080023805848FFF713FF5748FFF734FF5548FFF73C
S3150800239020FF08208DF8000000208DF80100272076
S315080023A08DF8020069208DF803005B208DF8040083
S315080023B045208DF805009DF800004C4908709DF8E9
S315080023C001004A4948709DF80200484988709DF8FE
S315080023D003004649C8709DF80400444908719DF8F1
S315080023E005004249487113BD08210170002141705A
S315080023F0272181706921C1705B21017145214171D5
S31508002400704738B50024374800F02AFF0500002D2C
S3150800241009D040F2F550854205D22A0034493148A0
S3150800242000F0E9FE2C00200032BD80B53148008856
S3150800243000284FD02F48008840F2F551884249D2EB
S315080024402848FFF7BEFE002803D02648FFF7E3FE1C
S3150800245040E02448FFF7EAFE002103E0244A525CE4
S315080024604254491C234A12889142F7D321480188CD
S315080024701C48FFF7E2FE1B4890F82600194981F828
S31508002480280018484069174991F826104901154A45
S315080024905269144B93F826305B01D25852F0004229
S315080024A04250104890F82600401C0E4981F8260034
S315080024B00C4890F826000B4991F82510884203D15C
S315080024C00020084981F826000020064908620548C8
S315080024D0FFF7A1FE01BD000040400050008F0248F2
S315080024E0008202484080FE1F9C5000084891FE1F4B
S315080024F0A480FE1F9691FE1F80B500F00DF81048C7
S315080025001049086000201049086005200F49086036
S3150800251000200F49086001BD00200C49086070477B
S315080025200A480068C00304D509480068401C0849E1
S315080025300860704780B5FFF7F3FF0548006802BDDD
S315080025407F32020014E000E018E000E010E000E04E
S315080025506491FE1F80B501201849087000F023F821
S3150800256000F001F801BD80B501F03EF8012813D04E
S315080025701248007801280FD1FFF7DCFF10490968D7
S31508002580104A1268511811F5FA71884204D30020CE
S315080025900A49087001F03EF801BD0949086070470C
S315080025A007480068704780B504480078012803D1B9
S315080025B0FFF7C0FF0349086001BD0000A291FE1F96
S315080025C05491FE1F5091FE1F0020DFF86814087012
S315080025D00020DFF8601488640020DFF8581481F8BA
S315080025E043000020DFF84C14A1F844000020DFF86F
S315080025F0441488700020DFF83C1448707047DFF8F0
S3150800260034040078002801D1002000E0012070473A
S315080026100020DFF8201481F84300704780B5017860
S31508002620FF291ED100F095F8DFF8080490F843005A
S31508002630012802D1102000F082F8DFF8F803B0F97B
S31508002640440001280CDB0120DFF8E81381F8430079
S31508002650DFF8E003B0F94410DFF8DC0300F053F8C4
S3150800266001BDDFF8D013097801294BD10178C929B2
S3150800267032D0CC293FD0CF293AD0D0292FD0D12952
S3150800268033D0D2292ED0F32917D0F4290FD0F52923
S315080026900AD0F6290ED0FA2912D0FC2913D0FD2922
S315080026A014D0FE2915D029E000F0D5F8BCE700F0D3
S315080026B0F5F8B9E700F0C4F8B6E700F015F9B3E79E
S315080026C000F0A6F8B0E700F09EF8ADE700F083F852
S315080026D0AAE700F072F8A7E700F039F9A4E700F0D6
S315080026E058F9A1E700F017F99EE700F084F99BE78F
S315080026F000F095F998E700F0A7F995E7202000F093
S315080027001EF891E7ACE780B589B200F022FF01BD5B
S31508002710F8B504000D001600002704E02078C71954
S31508002720641C00F055FE2800451E0028F6D1FFB2AD
S3150800273037600120F2BD0020BE4948707047FE216F
S31508002740BC4AD170BB4908710220BA49A1F84400B5
S31508002750704780B5FFF7EFFF0120B6490870FF20E4
S31508002760B449C8700020B3490871B248007950F0DE
S315080027701000B04908710020AE494871AD4840794B
S31508002780AC49487100F006FFAA49887100F017FFA6
S31508002790A849C87100F013FF80B2000AA54908725B
S315080027A00120A44948720120A24988720820A1493B
S315080027B0A1F8440000F067FF01BD80B500209D49DF
S315080027C00870FFF7B8FFFF209A49C8700120994999
S315080027D0A1F8440001BDFF209649C870002095491C
S315080027E00871944840789349487100209149887146
S315080027F000209049C87100208E49087206208D492C
S31508002800A1F84400704780B50020FFF798FF01BD86
S31508002810FF208849C8708948864988640020854908
S315080028200871002083494871002082498871072071
S315080028308049C1F8070008207E49A1F8440070477E
S31508002840FF217C4AD17040687A4988640120794919
S31508002850A1F84400704710B5040000F09BFE80B252
S31508002860401E6178884203DA2220FFF768FF14E0E9
S315080028706278734892B26F49896C00F0F3FEFF20C4
S315080028806C49C8706B48806C6178401869498864DF
S315080028906078401C6749A1F8440010BD10B50400D3
S315080028A000F078FE80B2401E6178884203DA222062
S315080028B0FFF745FF17E060685E49886462786048FC
S315080028C092B25C49896C00F0CDFEFF205949C87068
S315080028D05848806C61784018564988646078401C6E
S315080028E05449A1F8440010BD80B5FF21514AD17062
S315080028F0544A41684F48806CFFF70AFF4D490871F2
S3150800290000204C49487100204A49887108204949E5
S31508002910A1F8440001BD80B5FF204649C8700020D3
S315080029204449087100204349487100F033FE414983
S31508002930887100203F49C87100203E49087200206E
S315080029403C49487207203B49A1F8440001BD10B52F
S31508002950040000F01FFE621C80B2411E3548806CE0
S3150800296000F095FE002803D13120FFF7E8FE0FE0BE
S31508002970FF203049C87000F00DFE2E49896C80B2E0
S31508002980401E40182B49886401202A49A1F84400B2
S3150800299010BD10B5040000F0FDFD80B2801E617800
S315080029A0884203DA2220FFF7CAFE23E0FF202149E6
S315080029B0C87001201F49A1F844006078002807D193
S315080029C000F075FE002802D13120FFF7B8FE11E0AD
S315080029D0A21C61781748806C00F059FE002803D1C4
S315080029E03120FFF7ACFE05E01248806C617840188C
S315080029F01049886410BD80B541680E48806C00F0A7
S31508002A004AFE002803D13120FFF799FE06E0FF2091
S31508002A100849C87001200749A1F8440001BD80B5DE
S31508002A2000F0F8FDFF200349C87001200149A1F80C
S31508002A30440001BDB88FFE1FBB8FFE1FAC500008B7
S31508002A40BC8FFE1FBF8FFE1F80B53120FFF777FEB4
S31508002A5001BD000010B5DFF8FC030078401CDFF864
S31508002A60F41308700020DFF8E413087020E0DFF89C
S31508002A70E003DFF8D81309780C22514300EB010470
S31508002A8020886188084300280BD0DFF8C80300783F
S31508002A90A17A401A782804DB042100222000FEF7D8
S31508002AA0A3FEDFF8A8030078401CDFF8A01308701F
S31508002AB0DFF8980300780828D9DB10BD70B50C003C
S31508002AC0DFF88C530021DFF88423117006E0DFF865
S31508002AD07C130978491CDFF874231170DFF86C132E
S31508002AE00978082921DADFF86813DFF860231278F5
S31508002AF00C235A4301EB020529880029E7D0698887
S31508002B000029E4D001882A889142E0D141886A8860
S31508002B109142DCD106222E1D21003000FFF700FB72
S31508002B20DFF830030078A8726BE00021DFF81C2379
S31508002B30117006E0DFF814130978491CDFF80C2336
S31508002B401170DFF80813097808290EDADFF8001380
S31508002B50DFF8F82212780C235A4301EB020529887C
S31508002B600029E7D169880029E4D1DFF8E01209785D
S31508002B70082938D10021DFF8E02211700021DFF89A
S31508002B80DC2211700021B14A11701DE0B049AF4A2C
S31508002B9012780C235A4301EB0205AF490978AD4A6E
S31508002BA01278AB7AD21A914209DAAA490978AA7A2E
S31508002BB0891AA94A1170A5490978A84A1170A34922
S31508002BC00978491CA14A1170A04909780829DDDB52
S31508002BD0A24909789D4A11709D499C4A12780C238E
S31508002BE05A4301EB0205042201002800FFF798FA70
S31508002BF006222E1D21003000FFF792FA954800782C
S31508002C00A87270BD10B5964800882A2803D20020FD
S31508002C10934908805FE00020914908809148808A9E
S31508002C20B0F5807F03D0B0F5007F44D053E08D48DF
S31508002C30C08C8D49098888423CD18A48008D8A49CA
S31508002C404988884236D189498948FFF737FF4FF4C2
S31508002C5000708449888206228449864C2000FFF742
S31508002C605FFA06228449814C2000FFF759FA0622AA
S31508002C708149824C2000FFF753FA06227D49794C98
S31508002C802000FFF74DFA7748808B7649C884754847
S31508002C90C08B7449088574480088724988837248CD
S31508002CA040887049C8834FF4C1606E4988812A20DC
S31508002CB06B4908800FE06B48C08C6B4909888842CD
S31508002CC009D16848008D68494988884203D167490F
S31508002CD06748FFF7F3FE10BD10B55D486149C98B1B
S31508002CE0674A128891420CD15E49098C644A528817
S31508002CF0914206D1062263495A4C2000FFF710FA82
S31508002D0093E05849C98B604A12881140564A12887E
S31508002D105D4B1B881A4091420BD15249098C5A4A7D
S31508002D2052881140504A5288574B5B881A40914244
S31508002D3008D056490988564A118054494988544A40
S31508002D40518007E04749C98B514A11804549098C8A
S31508002D504F4A518000213D4A117004E03B490978E9
S31508002D60491C3A4A11703949097808290FDA38484E
S31508002D70364909780C22514308444549098802888E
S31508002D809142EBD14249498842889142E6D12F497E
S31508002D900978082943D10621FF22324C2000FEF784
S31508002DA023FD06210022334C2000FEF71DFD0622D6
S31508002DB03149324C2000FFF7B3F906222E492B4C35
S31508002DC02000FFF7ADF9324800882649C884304804
S31508002DD0408824490885244800882249888322484F
S31508002DE040882049C8834FF480701E4988824FF472
S31508002DF080701C49C88108201A490882062019498A
S31508002E00887404201749C8744FF4C160154988812D
S31508002E102048214908602A201149088013E0062223
S31508002E20011D104C2000FFF77BF906221249134CAE
S31508002E302000FFF775F908200A49888108480088A4
S31508002E400E300749088010BD00000000AA91FE1F39
S31508002E50588FFE1FAC91FE1FAD91FE1FAB91FE1F52
S31508002E609691FE1FA480FE1F6C91FE1FBA80FE1F5E
S31508002E70C080FE1FC480FE1F4891FE1FAA80FE1F49
S31508002E80C4500008A45000087491FE1F7091FE1FDC
S31508002E909091FE1FDA80FE1F7891FE1F0300002026
S31508002EA013F0030F09D0521E22BF13F8010B11F8B5
S31508002EB001CBB0EB0C00F3D07047121F22BF53F8BA
S31508002EC0040B51F804CB6045F7D0121D0AD200BA9C
S31508002ED09CFA8CFCB0EB0C0038BF6FF0000088BF82
S31508002EE001207047521E22BF13F8010B11F801CBBF
S31508002EF0B0EB0C00F6D0521C08BF1046704710B550
S31508002F000400616000F0DDFB206010BD10B5040010
S31508002F1000F0D7FB2168401A6168884201DB01206E
S31508002F2000E00020C0B210BD70B4C9B28B1000EB2F
S31508002F308303C9B28C1000EB84042469F82511F0C8
S31508002F400306F6B2F600B540AC431C61436F032492
S31508002F504D00AC40A3434367224B984202D0224B14
S31508002F60984205D1036E01248C40A343036624E0EE
S31508002F7053688B404360C9B2CB1000EB8303C9B2D8
S31508002F80CC1000EB8404246C072511F00706F6B272
S31508002F90B600B540AC431C64C9B2CB1000EB830342
S31508002FA0C9B2CC1000EB8404246C157A11F007061C
S31508002FB0F6B2B600B5402C431C64C9B28B1000EBC0
S31508002FC08303C9B28C1000EB84000069127811F0F3
S31508002FD00301C9B2C90012FA01F10843186170BCAD
S31508002FE070470000008E0248008F024870B4C9B2CC
S31508002FF08B0800EB8303C9B28C0800EB84042469B0
S31508003000F82511F00306F6B2F600B540AC431C618C
S31508003010C9B28B0800EB8303C9B28C0800EB8400A5
S315080030200069D2B211F00301C9B2C90012FA01F15E
S315080030300843186170BC704730B4436F03244D00D1
S31508003040AC40A3434367436FD2B2490012FA01F179
S315080030501943416730BC704701684FF4805289585C
S3150800306051F0010102684FF48053D15001684FF4C2
S3150800307080528958C907F9D4704701680B640068FB
S3150800308042647047DFF810030068DFF81013096818
S3150800309011F001018840704780B5FFF7F3FF40083B
S315080030A002BD38B50400200000F026F92000FFF71D
S315080030B0D3FF200000F0EBF80500D4E90223200036
S315080030C0FFF7DBFF4FF480602168086080202168E5
S315080030D08861DFF8CC02216841F218028850DFF8CF
S315080030E0C40221684FF480528850200000F021F86D
S315080030F0200000F052F85FF0FF30216841F2140218
S3150800310088507FF07C402168C1F810017FF07C4030
S315080031102168C1F80C017FF0C0202168C1F80002BF
S315080031204FF402702168C863002020622800C0B2EC
S3150800313032BD10B4002122E05FF0004203694C0161
S315080031401A5102694B011A4444F2F4535360026956
S315080031504B011A44836940F2F45404FB01F42344F6
S3150800316093604A1C90F824309A4200D100220369E1
S315080031704C012344046952012244DA60491C90F840
S3150800318024209142D8D30169026841F20C03D15038
S31508003190002180F8271010BC704710B400211CE0ED
S315080031A0DFF8042243694C011A5142694B011A445B
S315080031B0C36940F2F45404FB01F4234493604A1CA7
S315080031C090F825309A4200D1002243694C012344E5
S315080031D0446952012244DA60491C90F8252091423C
S315080031E0DED34169026841F21003D150002180F80C
S315080031F0261010BC704770B504000E001500206933
S3150800320094F827104901084481682A003000FEF71F
S3150800321087FF206994F8271049015FF00042425061
S3150800322094F82700401C84F8270094F8270094F89F
S315080032302410884202D1002084F82700206841F231
S3150800324014014058000609D58020216841F214026D
S3150800325088500020216841F208028850280070BD75
S315080032600021016990F8270040010858002801D577
S3150800327000210AE010F40341B1F5407F02D05FF067
S31508003280FF3102E0C0F30D40011F0800704710B57A
S315080032900400FFF701FF0100002022681032DFF862
S315080032A00C31994202D20821116023E0DFF800317F
S315080032B0994202D20C2111601CE0DFF8F8309942DD
S315080032C002D20021116015E0DFF8EC30994202D2F3
S315080032D0042111600EE0DFF8E430994202D2102191
S315080032E0116007E0DFF8D830994202D21421116044
S315080032F000E00220C0B210BD80B5042000F0FDF940
S31508003300DFF8C00000F0FEF9DFF8B80000F0E2F9D7
S3150800331001BD10B40468246914F03C04C9B254EA27
S31508003320C121D2B251EA821151F00101026811613C
S31508003330002102681269D20704D40068406918801F
S31508003340002005E0491C4FF6FF729142F1D3022096
S3150800335010BC704710B49BB20468636103681B69AC
S3150800336013F03C03C9B253EAC121D2B251EA821121
S3150800337051F0030102681161002102681269D2073F
S3150800338001D4002005E0491C4FF6FF729142F4D3A0
S31508003390022010BC70470000C091FE1F1046005066
S315080033A0040020028020010200001030C10E16021F
S315080033B00187930301E1F50581D1F00801C2EB0B02
S315080033C081B2E60E0400002080B500F0C3F901BD05
S315080033D080B500F0C4F901BD38B504000D000DF143
S315080033E0020302222900C9B22000FFF792FF002833
S315080033F018D16B4603222900C9B22000FFF789FFBE
S3150800340000280FD1BDF80200222809D1BDF8000016
S315080034104FF6F0710840B0F5AB5F01D1002002E02D
S31508003420032000E00420C0B232BD70B504000D00D0
S3150800343016002900C9B22000FFF7CEFF002826D1C2
S315080034402900C9B2200000F023F800281FD1002364
S31508003450B6F90200B0F5804F01D153F40053B6F91E
S315080034600400B0F5006F01D153F48073B0790028D9
S3150800347001D053F48053F079002801D053F48043E7
S315080034809BB200222900C9B22000FFF763FF70BD76
S3150800349038B504000D004FF4004300222900C9B2D4
S315080034A02000FFF757FF00280AD16B4600222900A3
S315080034B0C9B22000FFF72DFFBDF800100904F4D4A7
S315080034C032BD80B56B460122C9B2FFF722FFBDF8AF
S315080034D00000C0B2800810F0010002BD80B5FFF7F9
S315080034E073F800F066F901204649087000F099FA69
S315080034F000204449087001BD80B56946424800F07D
S315080035003AFA012807D101203E4908709DF80010B3
S315080035103D48FFF783F869463B4800F0DAFA012888
S3150800352007D10020374908709DF800103648FFF784
S3150800353075F869463448FEF71BFA012807D10320B7
S31508003540304908709DF800102F48FFF767F801BD4D
S31508003550704738B504000D002A480078012804D1C0
S315080035602900C9B2200000F0DAF9264800780028B8
S3150800357004D12900C9B2200000F07EFA214800785B
S31508003580032804D12900C9B22000FEF7C9F9FFF7BC
S315080035903FF831BD1B480078002805D0022807D01F
S315080035A004D3032806D007E0402006E0082004E0FC
S315080035B0002002E0402000E0402080B27047114819
S315080035C00078002805D0022807D004D3032806D09F
S315080035D007E0402006E0082004E0002002E0402042
S315080035E000E0402080B2704780B5FFF708F802BDBA
S315080035F080B5FEF78AF9032002490870FEF7D3FF63
S3150800360001BD0000A080FE1F4890FE1F80B500F097
S31508003610F9FA01BD10B500F042F8002802D1FFF70B
S31508003620E7FF19E000F087F8002802D1FFF7E0FF6E
S3150800363012E0FFF78DFFFEF76FFF00F034F8074939
S3150800364008400749086000F02EF8001D046800F0DD
S31508003650DBFAA047FFF7CCFF10BD000080FFFF1F75
S3150800366008ED00E070B504000D00160005E02878A6
S3150800367020706D1C641CFFF7ABFE3000461E80B23E
S315080036800028F4D170BD80B500F0C6FA01BD80B53A
S3150800369000F0CDFA02BD80B500F007FB02BD80B58B
S315080036A000F073FB02BD80B500F0BCFB02BD80B51F
S315080036B000F029FB002801D1002001E000F097FB6B
S315080036C002BD80B5FEF736FF02BD0000DFF84800F0
S315080036D000687047010F20F07040DFF840200C2387
S315080036E059435050704780B5FFF7F0FFDFF83010A8
S315080036F0096811F00101C84002BDC0B2DFF8241004
S3150800370008607047010F20F07040DFF81C200C237A
S315080037105943505070470000C091FE1F1444005092
S31508003720144600500446005048460050406AC840B7
S3150800373010F00100704780B50D210548FFF7F6FF28
S31508003740002801D1002002E000F0FEFC012002BDA5
S31508003750008F024880B5642000F0CEFC01BD80B51C
S3150800376000F0CDFC01BD0000016851F04001016088
S315080037707047016831F0400101607047016851F0F7
S3150800378001010160704701684908490001607047F6
S315080037900068C06970470068C1617047816851F068
S315080037A0005181600168C96851F000510068C16024
S315080037B0704710B584B0FFF796FF040002E0640076
S315080037C0FFF706FE80488442F9D38048844203D333
S315080037D06408FFF7FDFDF8E7220001217C4800F0A8
S315080037E0B3FD00947B4801904FF4FA50ADF80800F9
S315080037F00120ADF80A0069467748406800F0DAFC0F
S3150800380075484068FFF7B0FF73484068FFF7B6FF92
S3150800381072487349086002207149496860F39F71CC
S315080038206F48416040F2E17020F000406C494968F9
S3150800383060F31C016A4A51606949896860F31C0192
S31508003840674881606648406830F0005064494860BF
S315080038506348FFF7A3FF082061490873002005E0C5
S3150800386000215F4AC0B202441174401C01005C4A40
S31508003870127BC9B29142F3D30120594908765848B8
S3150800388000F0BFFD00220121514800F029FD5548EE
S315080038905549086002205449496860F39F715248A7
S315080038A0416040F2676020F000404F49496860F384
S315080038B01C014D4A51604C49896860F31C014A480D
S315080038C081604948406830F000504749486046489A
S315080038D0FFF764FF082044490873002005E000212B
S315080038E0414AC0B202441174401C01003E4A127B90
S315080038F0C9B29142F3D300203B4908763A4800F012
S3150800390080FD01220121324800F0EAFC3248406875
S31508003910FFF72FFF30484068FFF735FF1FBD10B58A
S315080039202F4A1173002106E0C9B2425C2C4BC9B27A
S315080039300B441A74491C0A00294B1B7BD2B29A42C3
S31508003940F2D3274800F0B7FD02212548FFF723FFE9
S31508003950234800F0D1FDFEF7EDFD10F132042048B2
S31508003960FFF716FF800705D5FFF732FDFEF7E2FDE4
S315080039708442F4D210BD70B504000E0000251A4822
S31508003980FFF706FFC0071BD5174800F0CEFD002835
S3150800399012D11548007B3070002007E01249C0B2EA
S315080039A00144097CC0B221540125401C01000E4A7D
S315080039B0127BC9B29142F1D301210B48FFF7EBFE06
S315080039C02800C0B270BD0000001BB700010E270713
S315080039D00040014820A107007080FE1F00500148E2
S315080039E00091FE1F205001482091FE1FD0F81401B7
S315080039F0000B10F001007047D0F8140110F4407065
S31508003A007047C0F818117047D0F81401C00810F0B4
S31508003A1001007047016C0909090151F002010164AE
S31508003A207047E0B54FF46140009008208DF8040017
S31508003A3008208DF8050001208DF8060010208DF865
S31508003A4007000020ADF8080069466748006800F0DE
S31508003A50A7FD0123042210216348006800F069FECF
S31508003A600123042200216048006800F077FE5E48C2
S31508003A700068FFF7CFFF07BD70B504000D00EDB273
S31508003A80412D03DB7A21594800F0BCFE2800C0B25C
S31508003A9000F07EF8C0B2012803D07E21534800F01A
S31508003AA0B1FE00260DE0FFF793FCB6B2A05D00F06C
S31508003AB06FF8C0B2012803D087214C4800F0A2FE57
S31508003AC0761C30002900C9B280B289B28842EAD38E
S31508003AD070BD38B504000D0045480078002817D198
S31508003AE0444800F044F801283FD1424800780028AD
S31508003AF03BD040480078412837DAFEF71BFD3E499F
S31508003B00086000203D4908700120394908702CE0FA
S31508003B1038483A4909780844401C00F028F8012832
S31508003B2019D136480078401C344908703348007863
S31508003B3030490978884218D13048027892B230491B
S31508003B402000FFF78FFD0020294908702B480078D0
S31508003B50287001200AE0FEF7EDFC27490968643160
S31508003B60814202D2002022490870002032BD10B5D9
S31508003B7004001D480068FFF747FF002806D11A48C9
S31508003B80006800F064FD2070012000E0002010BDF0
S31508003B9038B50400012514480068FFF727FF0028F8
S31508003BA001D000201FE0E4B2210089B20E48006867
S31508003BB000F033FDFEF7BEFC10F10A040A4800685F
S31508003BC0FFF71AFFC00506D4FFF702FCFEF7B2FCA2
S31508003BD08442F3D200254FF4807103480068FFF74A
S31508003BE010FF2800C0B232BD8880FE1F044F0008AF
S31508003BF0A691FE1F0490FE1F6891FE1FA591FE1F49
S31508003C000590FE1F72B6704762B6704780B500F021
S31508003C102AFE10F0010002BD5FF0FF30DFF8B8148D
S31508003C2008605FF0FF30DFF8B4140860704770B5BD
S31508003C3006000C001500300000F054FA0600DFF804
S31508003C40A004D0F89C00DFF89814D1F8A010081842
S31508003C50401E801B611E884201D2002024E03000ED
S31508003C6000F0EEF9FF2805D0A019401E00F0E8F98B
S31508003C70FF2801D1002017E0B00A4FF480614843BD
S31508003C80DFF85C140968884207D123002A0031004E
S31508003C90DFF8480400F0FBF806E023002A003100AC
S31508003CA0DFF8340400F0F3F870BD70B505000C00B9
S31508003CB0280000F017FA0500DFF82404D0F89C0065
S31508003CC0DFF81C14D1F8A0100818401E401B611E0E
S31508003CD0884201D2002015E0280000F0B1F906005C
S31508003CE06019401E00F0ACF9F6B2FF2E02D0C0B241
S31508003CF0FF2801D1002005E00100C9B23000C0B29A
S31508003D0000F051F970BD80B500200090DFF8CC03B3
S31508003D10006810F1010F01D1012035E00098DFF8A5
S31508003D20BC134968081800900098DFF8B013896832
S31508003D30081800900098DFF8A413C96808180090BE
S31508003D400098DFF898130969081800900098DFF8BA
S31508003D508C134969081800900098DFF88013896960
S31508003D60081800900098DFF87413C96908180090BD
S31508003D700098C04300906A460421DFF8640300688F
S31508003D8010F50070FFF753FF02BD0020DFF850134F
S31508003D90096809680818DFF848130968091D0968D9
S31508003DA00818DFF83C130968083109680818CC496F
S31508003DB009680C3109680818C94909681031096881
S31508003DC00818C7490968143109680818C4490968F0
S31508003DD0183109680818C043C149096811F5007106
S31508003DE00968884201D1012000E00020704780B5AB
S31508003DF0BA48006810F1010F06D0B84800F08AF8F2
S31508003E00002801D100200CE0B348006810F1010F2A
S31508003E1006D0B14800F07EF8002801D1002000E065
S31508003E20012002BDAE480068704780B58A0501D0FA
S31508003E3000200BE002688A4201D1012006E00160F9
S31508003E404FF48062001DFFF70DFC012002BD38B556
S31508003E5004000D00A148844208D19F4C2900200087
S31508003E60FFF7E3FF002810D100200FE09C48006808
S31508003E70854203D1994C9A480568EFE7200000F07F
S31508003E8049F80028EAD1002000E0200032BD2DE9DB
S31508003E90F04104000F0015001E00B80A4FF48061B7
S31508003EA001FB00F8206810F1010F07D141462000F8
S31508003EB0FFF7BBFF002801D1002029E02068404514
S31508003EC008D041462000FFF7C2FF0400002C01D1AC
S31508003ED000201DE02068381A2044071DFFF778FAED
S31508003EE0201D381AB0F5806F0AD318F580612000B6
S31508003EF0FFF7ADFF0400002C01D1002008E0271DC4
S31508003F00287838707F1C6D1C761E002EE6D101209D
S31508003F10BDE8F0812DE9F0410400206800F090F832
S31508003F20FF2801D100203CE0002500E06D1C042D8F
S31508003F3036D2FFF74DFA20684FF4807101FB05066B
S31508003F404FF4807000FB05F02044071DFEF7F2FAD7
S31508003F5010F10D083900300000F088FC01E0FFF789
S31508003F6037FAFFF753FE002805D0FEF7E3FA804537
S31508003F70F5D2002015E000F076FC30F0100000289D
S31508003F8001D000200DE0002000E0401CFF28CDD81D
S31508003F90811909783A5CC9B29142F6D0002000E04E
S31508003FA00120BDE8F081F8B504000D0028002100C5
S31508003FB0C0B2C9B2884201D2002040E02000484978
S31508003FC0097AC0B2884206D3454890F8A400290069
S31508003FD0C9B2884201D2002031E000E0641C280002
S31508003FE02100C0B2C9B2884228D3FFF7F1F92000F0
S31508003FF0C0B200F051F8060016F1010F01D10020F9
S315080040001DE0FEF797FA00F5C857C837300000F0EC
S3150800401048FC01E0FFF7DCF9FFF7F8FD002805D0BA
S31508004020FEF788FA8742F5D2002008E000F01BFC6C
S3150800403030F020000028D1D0002000E00120F2BD99
S3150800404038B50400002500E06D1CEDB20E2D21D216
S31508004050FFF7BEF92248EDB20C2101FB05F14058E5
S315080040608442F1D31E48EDB20C2101FB05F14058FC
S315080040701B49EDB20C2202FB05F2114449680818E7
S315080040808442E1D21648EDB20C2101FB05F1084441
S31508004090007A00E0FF2032BD70B506005FF0FF34FD
S315080040A0002500E06D1CEDB20E2D12D2FFF790F937
S315080040B00B48EDB20C2101FB05F10844007A3100EA
S315080040C0C9B28842EED10648EDB20C2101FB05F1D2
S315080040D04458200070BD0000E886FE1FEC8AFE1FCB
S315080040E05C4E0008010E082901D110F18060704766
S315080040F012FA01F14160704717490880704780B588
S31508004100FEF718FA1549096888421CD3144800783E
S31508004110002808D1012012490870012209211148F6
S31508004120FFF7E6FF08E000200D4908705FF48032CB
S3150800413009210C48FFF7DCFFFEF7FCF90649098858
S3150800414040180649086001BD80B55FF48032092130
S315080041500448FFF7CDFF01BD9491FE1F5891FE1F3D
S31508004160A391FE1F00850248D0F8C40110F4407FD1
S3150800417001D1012000E00020C0B27047C9B2D2B216
S3150800418051EA0241DBB251EA0361C0F8C411704733
S31508004190016851F0400101607047016831F0400143
S315080041A001607047814200D308007047884200D3F7
S315080041B0080070472DE9F04104000D000C220C227E
S315080041C0002601275FF00008002042F21071012244
S315080041D000E0521C412A40D22B685FF00A0C0CFB07
S315080041E003F3B3FBF2FC6B68BCFBF3F35FF00A0E58
S315080041F0B3FBFEF80EFB183EBEF1060F05D35FF0C3
S315080042000A0EB3FBFEF35B1C03E05FF00A0EB3FB7A
S31508004210FEF3002B06D05FF00A0E0EFB03FEBCFB76
S31508004220FEFC03E00A23BCFBF3FC0123D5F804E0FB
S31508004230F44504D3D5F804E0BCEB0E0C03E0D5F83E
S3150800424004E0BEEB0C0C152BC3D28C45C1D216006C
S3150800425018006146BCF57A7FBBD242F21071402243
S3150800426000E0521E032A1BD3531C42F2107C0CFB9F
S3150800427003F3B3FBF0F3B5F808C0634504D3B5F808
S3150800428008C0B3EB0C0C03E0B5F808C0BCEB030C94
S315080042908C4501D217006146B5F808C06345E0D2DF
S315080042A0C01BB0F101082000FFF772FFB8F101004A
S315080042B0000310F4E0406989491E890111F0C00124
S315080042C00843791E090211F470610843711E11F042
S315080042D03F01084320612000FFF75FFFBDE8F0813A
S315080042E070B504000D0016002000FFF73DFF0028FA
S315080042F0FAD06B1CDBB23200D2B202212000FFF7E3
S315080043003DFF70BD10B50400DFF87402FFF7FAF937
S31508004310DFF86C02FFF7DEF92068400840002060ED
S3150800432020688007FCD410BD80B500F065F8012828
S3150800433002D0022803D005E0FFF7D5F903E000F024
S31508004340C7FA00E0002002BD2DE9F04104000E0086
S3150800435015002000FFF7D6FF3100C9B2200000F093
S3150800436042F82000FFF7E0FF8046B8FBF5F0D0F5ED
S3150800437080610020FFF716FF40F2FF31FFF716FFB6
S315080043800600D6F58060B8FBF0F7A8095FEA98182A
S3150800439040F2FF314FF480625043B0FBF8F0FFF76C
S315080043A005FF00FB08F1890A8901691AEA1B91428F
S315080043B001D3012100E00021C9B2002900D106007D
S315080043C0C9B2002901D0012000E00220E168DFF827
S315080043D0B4211140E160E168C0B256EA8030084372
S315080043E0E060BDE8F081D0F8C82112091201C9B20F
S315080043F01143C0F8C8117047D0F8C80110F00F0073
S31508004400704710B504002068DFF87C1108184009C9
S315080044104109000210F4F85050EA413021688968D1
S3150800442031F47F41226891602168896808432168D0
S3150800443088606068C0F34070C00704D56068C0F340
S315080044404070C00736D5207E002802D0207E01287D
S3150800445030D120202168C8616068C0F34070002808
S3150800446010D1606810F06040616850EA81402168A8
S315080044708861A06810F06040A16850EA8140216810
S31508004480C86005E0606821688861A0682168C8601E
S31508004490207E012807D1200000F00DF85FF00060AB
S315080044A02168C86103E04FF400602168C861374895
S315080044B02168C86110BD0321017E012918D1202178
S315080044C00268D1610168096831F07061027B1206E1
S315080044D012F0706211430268116001690268116185
S315080044E04169026851612A490068C161002100E0FA
S315080044F003210800C0B2704701210168C969C1F3E8
S3150800450040110268D269C2F30022002901D10421B0
S3150800451008E0012A01D1022104E05FF0E0610068A9
S31508004520C16100210800C0B27047012100210022A4
S315080045300168C969C1F3C0210268D269C2F3800261
S31508004540002901D0032118E0012A01D1022114E033
S315080045500168096901610168496941610168C969B8
S31508004560C1F380010268D269C2F3C002C9B2002948
S3150800457002D0D2B2002AEBD100210800C0B270479F
S3150800458010000010003CFFFF00B0FEB74000A00678
S3150800459040002800806B10F080007047C1647047A7
S315080045A070B504000D001026200000F05BF8E879CD
S315080045B0002800D0EE7932002968200000F07BF848
S315080045C0A879401EB11CC901090A090251EA40002E
S315080045D040F4403050F00100E0632879401E0006A0
S315080045E050F4817060636879002806D0606B697939
S315080045F0491E50EA0140606305E0606B2979491E4F
S3150800460050EA014060634FF4A060A0635FF0FF309A
S31508004610E064B5F90800206470BD38B504000D00E3
S31508004620D4F8080110F0E06F0DD12000FFF7B2FFB3
S315080046308028FAD04FF400512000FFF7AFFFADB243
S31508004640C4F8805002E0ADB2C4F8805131BDD0F84C
S315080046500C1111F0E06F01D1406D01E0D0F81C019A
S3150800466080B2704710B504005848844202D05848B2
S31508004670844203D1574800F088F812E0564884422D
S3150800468002D05648844203D1554800F07EF808E027
S315080046905448844202D05448844202D1534800F018
S315080046A074F80320E060E068C007FCD5206C0009B8
S315080046B00001206410BDF8B504000E001500642E34
S315080046C034D3002D32D0FFF70EF86421B0FBF1F198
S315080046D06420B6FBF0F60123012040F2FF3E40F2CB
S315080046E0FF3212E002FB01F705FB06FCB7FBFCF7FD
S315080046F05FEA972CBF05BF0DBCF5806F04D27745DE
S3150800470002D2BE4660461300521E002AEAD153F46E
S31508004710004121616169364A11406A1E51EA8221C7
S31508004720401E51EA00406061002000E00120C0B24E
S31508004730F2BD30B4D0F8084134F0E064C0F808415E
S31508004740D0F808412B4D2C4054EA03231943D2B222
S3150800475051EA0261C0F8081130BC704730B4D0F88D
S315080047600C4134F0E064C0F80C41D0F80C41224DFD
S315080047702C4054EA03231943D2B251EA026151F09C
S315080047808051C0F80C1130BC704780B51149884279
S3150800479008D14FF40060FEF7B5FF4FF40060FEF74E
S315080047A099FF12E00E49884206D11448FEF7AAFF7F
S315080047B01248FEF78FFF08E00C49884205D11048D9
S315080047C0FEF7A0FF0E48FEF785FF01BD0000034077
S315080047D000020340080003400000024800020248A5
S315080047E008000248004002480042024808400248C1
S315080047F0EF8000FCC0C0FFF8C0C0FFEF80000010CB
S315080048000001001080B5FEF7E3FDFCE72B485021B8
S31508004810016070472A4A10602A4A11607047274982
S31508004820AA220A60284955220A602449A0220A6059
S315080048300100AA20086070472049AA220A60224976
S3150800484055220A601D4980220A601C49AA220A606C
S315080048501D4955220A600100302008607047174834
S31508004860F5210160704719480068704770B5040063
S315080048700D00FFF7F4FFFFF7C9FF002607E005EB79
S315080048808600416855F82600FFF7C4FFB61C402E7F
S31508004890F5D32000FFF7C3FF0C480068C007FBD418
S315080048A070BD10B50400FFF7DAFF2000FFF7C4FF5C
S315080048B006480068C007FBD410BD00005455000C1C
S315080048C0F055000CF455000CA8AA000C102000584E
S315080048D000487047001BB70080B566480068C007E7
S315080048E009D46548006850F00100634908606148CA
S315080048F00068C007FBD561480068800509D560488F
S31508004900006850F400705E49086041F64C5000F0AB
S31508004910EBF85C48006850F400205A49086040F6F5
S31508004920C41000F0E1F8574800685749084055494F
S3150800493008605648006810F0300F24D053480068C5
S315080049405349084051490860FFF7C2FF4F490968B3
S31508004950504AB0FBF2F0401E51EA00404B4908604D
S315080049604D480068400840004B49086045480068C3
S3150800497030F40030434908604848006810F4607015
S31508004980B0F5607FF8D13F48006850F001003D4916
S3150800499008603C48006850F010003A4908604048F2
S315080049A0404908603748006850F0400035490860BB
S315080049B03448006830F01000324908603148006811
S315080049C050F480202F490860344800684007FBD51A
S315080049D02C480068400840002A4908602F480068AB
S315080049E0C007FBD45FF001102F49086000202F494B
S315080049F0086000202E49086000202E490860002023
S31508004A002D49086003202D4908602D482D49086066
S31508004A102D482E4908601B48006830F040001949A7
S31508004A2008602B481F4908604FF4166000F05CF8D0
S31508004A3028481C4908604FF4616000F055F826487C
S31508004A40184908604FF4965000F04EF82348154967
S31508004A50086041F2707000F047F821481149086073
S31508004A604FF4E15000F040F800201E49086000F0BD
S31508004A7059F801BD0042005004420050004400505D
S31508004A800844005014470050FDFFFEFF044700503D
S31508004A90CFFFF0FFA02526001C4700501047005006
S31508004AA0002F0B01184700500C46005014460050C2
S31508004AB01046005020460050244600501C46005020
S31508004AC00500010018460050030020012846005042
S31508004AD0002F0501002F0301002F0201002F0101FD
S31508004AE0002F00010446005081B00021009103E028
S31508004AF000BF0099491C009100998142F8D301B082
S31508004B007047000010B510225FF00051044C2000D9
S31508004B10FDF706FB00F054F8FFF7DEFE10BD00BFF8
S31508004B20B091FE1F80B51F480068C00327D51E48F0
S31508004B300068C00701D51D4801E0FFF7C9FE1C49FA
S31508004B400968490713D51B490968C1F30361491C5C
S31508004B50184A1268C2F30622521C164B1B68C3F386
S31508004B6006435B1C5943B0FBF1F0504308E011497A
S31508004B70096811F07F014B1CB0FBF3F000E00B480D
S31508004B800849096801F0FF01491CB0FBF1F00A4920
S31508004B90096811F00101491CB0FBF1F007490860EA
S31508004BA001BD00BF0C4600501C47005000366E0180
S31508004BB0104700501847005010460050C091FE1F7D
S31508004BC072B60D480D490860BFF34F8F62B60C48A0
S31508004BD0006850F470000A4908600A48006830F016
S31508004BE0080008490860084800680009000150F0F4
S31508004BF004000549086070470000000808ED00E059
S31508004C0088ED00E014ED00E014200058026E012340
S31508004C1013FA01F132EA010101667047C9B200EBE5
S31508004C208103DB69DB08DB00D2B21A43C9B200EBA9
S31508004C308100C2617047C268D208D200C9B211F0B9
S31508004C4007011143C1607047016851F040010160D6
S31508004C507047016831F040010160704780B5002057
S31508004C608DF8000000F013F800F06EF800F0DEF89A
S31508004C706946002000F07CF89DF80000012801D163
S31508004C80FEF7B6FC00F013F800F0DEF8FCE780B596
S31508004C90802209212748FEF7A9F900220D21264876
S31508004CA0FEF7A4F90D212448FFF7B0FF01BD00B5B2
S31508004CB08DB000208DF818000120079002208DF88D
S31508004CC0200006AA04211D48FEF72EF990208DF82B
S31508004CD00C000120049002208DF8140003AA052177
S31508004CE01648FEF721F9012200211548FFF796FF1D
S31508004CF000208DF8240009AA0D211048FEF714F9A2
S31508004D0090208DF800000120019002208DF80800FF
S31508004D106A460C210948FEF707F90A48FFF794FF87
S31508004D2002210848FFF787FF0648FFF792FF0DB0F4
S31508004D3000BD000000850248008F02480081024835
S31508004D40000003400043014880B500F025F800281C
S31508004D500DD1344834490860002004E00021324A65
S31508004D6002441171401C3828F8D300F024F801BD1C
S31508004D7070B504000D00002600F00EF8002808D0D3
S31508004D80382C06D2002D04D02748204400792870F4
S31508004D9001263000C0B270BD10B500242248006854
S31508004DA02049884204D100F00CF8002800D00124DC
S31508004DB02000C0B210BD80B500F010F81A498887E7
S31508004DC001BD10B5002400F009F81749898F80B293
S31508004DD0884200D101242000C0B210BD002012492B
S31508004DE0096850FA81F010490968090A50FA81F0F1
S31508004DF00D490968090C50FA81F00B490968090E32
S31508004E0050FA81F0002105E0074A0A44127950FA5F
S31508004E1082F0491C3829F7D380B2C043401C80B2BF
S31508004E2070470000A2E742CE0080FE1F80B5FEF75D
S31508004E30EDFBFEF7C9FAFDF75FFBFEF724FCFEF76C
S31508004E404DFBFDF787FB01BD80B5FEF7C1FAFDF7FF
S31508004E5067FBFEF751FBFDF786FB01BD0080000CE2
S31508004E60004000000200000000C0000C00400000E6
S31508004E70030000000000010C0040000004000000D0
S31508004E800040010C00400000050000000080010CF5
S31508004E90004000000600000000C0010C00400000B1
S31508004EA0070000000000020C0000020008000000D5
S31508004EB00000040C00000400090000000000080CB3
S31508004EC0000004000A00000000000C0C00000400AA
S31508004ED00B0000000000100C000004000C0000008D
S31508004EE00000140C000004000D0000000000180C5F
S31508004EF0000004000E00000000001C0C0000040066
S31508004F000F000000433A5C576F726B5C736F6674F0
S31508004F10776172655C4F70656E424C545F584D43BD
S31508004F20343730305F6578747261735C54617267C8
S31508004F3065745C536F757263655C41524D434D34BD
S31508004F405F584D43345C756172742E63000000002F
S31508004F5019E050F8041BCB0744BFA9F101035918FF
S31508004F60121F0023042A41F8043BF9D25FEA827C27
S31508004F700B4604D54FF0000CA1F800C09B1CD107C6
S31508004F8044BF0021197050F8042B002AE1D170475C
S31508004F9010B450F8041B79B102684368024408301B
S31508004FA0DC0744BFA9F10104E31852F8044B43F89F
S31508004FB0044B091FF9D1ECE710BC704710B5074937
S31508004FC079441831064C7C44163404E00A68081DF6
S31508004FD0114488470146A142F8D110BD2C000000B3
S31508004FE0540000004EF68851CEF20001086840F4DD
S31508004FF070000860BFF34F8FBFF36F8F4FF00070DC
S31508005000E1EE100A7047000049FFFFFF0C1100008F
S31508005010A480FE1FA0300000000000200000000051
S3150800502071FFFFFF64000000580200004080FE1F69
S315080050300000000000F00BF8002801D0FFF7BEFFC3
S315080050400020AFF30080FFF709FE00F002F8012008
S31508005050704700F001B800000746384600F002F82D
S31508005060FBE7000080B5AFF30080024A1100182064
S31508005070ABBEFBE726000200DFF808D002488047EF
S3150800508002480047C899FE1F054B000891500008C2
S31508005090AFF30080FFF7A6FFFFF7CCFF0100004043
S315080050A000080000FFFFFFFFFFFF00004F70656E5E
S315080050B0424C5400ADDE122363825363FFFFFFFFA9
S315080050C000000000FFFFFFFFFFF7FEBFFFF7FEBF70
S315080050D0FFF7FEBFFFF7FEBFFFF7FEBFFFF7FEBFF6
S315080050E0FFF7FEBFFFF7FEBFFFF7FEBFFFF7FEBFE6
S315080050F0FFF7FEBFFFF7FEBFFFF7FEBFFFF7FEBFD6
S31508005100FFF7FEBFFFF7FEBFFFF7FEBFFFF7FEBFC5
S31508005110FFF7FEBFFFF7FEBFFFF7FEBFFFF7FEBFB5
S31508005120FFF7FEBFFFF7FEBFFFF7FEBFFFF7FEBFA5
S31508005130FFF7FEBFFFF7FEBFFFF7FEBFFFF7FEBF95
S31508005140FFF7FEBFFFF7FEBFFFF7FEBFFFF7FEBF85
S31508005150FFF7FEBFFFF7FEBFFFF7FEBFFFF7FEBF75
S31508005160FFF7FEBFFFF7FEBFFFF7FEBFFFF7FEBF65
S31508005170FFF7FEBFFFF7FEBFFFF7FEBFFFF7FEBF55
S31508005180FFF7FEBFFFF7FEBFFFF7FEBFFFF7FEBF45
S31508005190FFF7FEBFFFF7FEBFFFF7FEBFFFF7FEBF35
S315080051A0FFF7FEBFFFF7FEBFFFF7FEBFFFF7FEBF25
S315080051B0FFF7FEBFFFF7FEBFFFF7FEBFFFF7FEBF15
S315080051C0FFF7FEBFFFF7FEBFFFF7FEBFFFF7FEBF05
S315080051D0FFF7FEBFFFF7FEBFFFF7FEBFFFF7FEBFF5
S315080051E0FFF7FEBFFFF7FEBFFFF7FEBFFFF7FEBFE5
S315080051F0FFF7FEBFFFF7FEBFFFF7FEBFFFF7FEBFD5
S31508005200FFF7FEBFFFF7FEBFFFF7FEBFFFF7FEBFC4
S31508005210FFF7FEBFFFF7FEBFFFF7FEBFFFF7FEBFB4
S31508005220FFF7FEBFFFF7FEBFFFF7FEBFFFF7FEBFA4
S31508005230FFF7FEBFFFF7FEBFFFF7FEBFFFF7FEBF94
S31508005240FFF7FEBFFFF7FEBFFFF7FEBFFFF7FEBF84
S31508005250FFF7FEBFFFF7FEBFFFF7FEBFFFF7FEBF74
S31508005260FFF7FEBFFFF7FEBFFFF7FEBFFFF7FEBF64
S31508005270FFF7FEBFFFF7FEBFFFF7FEBFFFF7FEBF54
S3150800528000C0005000000000080027695B450000C8
S31508005290A02F00202030002000000020D01700207A
S315080052A000000000040400000000000000000000E8
S315080052B000420148004301480044014800450148AE
S315080052C00046014800470148000003400002034029
S315080052D00000024800020248004002480042024814
S309080052E004010000B7
S7050800509111
